:020000040000FA
:100000008A150A16612DFF3F682D0800FF3FFF3F4C
:10001000FF3FFF3FFF3FFF3FFF3FFF3FFF3FFF3FF0
:100020008A150A1600208A110A123126F012F212DD
:10003000F217C001C1018611701183120313F80178
:10004000F901FA01FB01FC01FD01FE01FF01203075
:1000500084007925A000243020020319FD283C30BB
:100060002002031D2928840AC9010230BD00792518
:10007000C907D6208000840ABD0B37282208C80093
:10008000210EC80406304802BD007925C907D620D4
:100090008000840ABD0B45280230BD007925D6209A
:1000A0008000840ABD0B4E287925BC003E303C02FE
:1000B000031D812884030008BC008403000EBC04D7
:1000C00049083C02031D8A28831324308400000859
:1000D000CA008403000ECA04CA0803197E284E30E1
:1000E0004A0203187E280611861590304A07073009
:1000F0000318013E8A004A0890271B280030BF00E1
:1001000099280130BF0099280230BF009928033098
:10011000BF0099280430BF0099280530BF009928F6
:100120000630BF0099280730BF0099280830BF006B
:1001300099280A30C8000030CA00831710308400A4
:100140003F08800006157015C8251B2841346C3403
:100150006C34203459346F34753472342034423462
:10016000613473346534203441347234653420345E
:10017000423465346C346F346E3467342034543414
:100180006F34203455347334FF3FFF3FFF3FFF3F50
:10019000F6308100D428EC308100D428D83081009A
:1001A000D4283D308100D4280B110800F700F60058
:1001B0000F30F605473077020318E4284130770204
:1001C000031CE4280930F60776080800B800B900D7
:1001D000F030B905390EF220B9000F303805F220A1
:1001E000B8000800F6000A307602031CFA283730FF
:1001F0007607FC283030760708000530BD00213036
:10020000840079258000840ABD0B0129BC000D30D3
:100210003C02031D7E2830307625323076251B289F
:100220000E30C8000130CA008A110A1600208A1157
:100230000A127015C82508001230C8000230CA0022
:1002400042267015C82508000E30C8000430CA00C8
:1002500070150230D5008A150A1607208A110A1275
:10026000711C35296024BF00E5247015C8250800DD
:100270000830C8000530CA0083132608BC00250ECC
:10028000BC04BC0803194529472958274829512788
:10029000C82508000830C8000630CA002608C20079
:1002A000250EC2042808C300270EC3042908C40071
:1002B0002A0EC404C82508000A30C8000730CA0046
:1002C0008A110A160C208A110A127015C825080016
:1002D0000A30C8000830CA00A9267015C8250800D1
:1002E0000830C8000930CA002608C100250EC10424
:1002F000C82508000830C8000A30CA002608BC001B
:10030000250EBC04F212BC0803198729F216C82571
:1003100008000830C8000B30CA002608BC00250EB3
:10032000BC04BC08031D9D299529F2178A110A16E1
:10033000D2218A110A12F217A429F2178A110A1679
:10034000D2218A110A12F213C82508000830C80009
:100350000C30CA002608BC00250EBC047213BC0871
:10036000031DB32972170B30D5008A150A16072012
:100370008A110A12C8250800080008008312031316
:10038000F016061008000830C8001230CA00C82550
:1003900008000830C8001B30CA008A110A16AA21BA
:1003A0008A110A120430D500922408000830C800CF
:1003B0001E30CA008A110A16AA218A110A120330B5
:1003C000D5006F2408000830C8002330CA008A1105
:1003D0000A16B0218A110A121C30D5006F240800B9
:1003E0000830C8002430CA008A110A16B0218A11C8
:1003F0000A121D30D500922408000830C8002530AC
:10040000CA00C8258A110A16D2218A110A120800C8
:100410000830C8002630CA008A110A1688218A11BD
:100420000A12C82508000830C8002730CA008A11FF
:100430000A168B218A110A12C82508000830C80044
:100440002830CA008A110A16D2218A110A12C82538
:10045000522C0830C8002930CA008A110A167921A6
:100460008A110A12C82508000830C8002A30CA00BC
:1004700083132608BE00250EBE048A110A16B32176
:100480008A110A12C82508000830C8002B30CA009B
:100490002608BC00250EBC0400303C0203195B2A70
:1004A00001303C0203196F2A02303C020319592A19
:1004B000822A1727822A17276425042764254927BB
:1004C0008719822A4127871587114927D120871943
:1004D000822A0B1D672A0730BF00E524822A1727CE
:1004E0006425042741278715871149271930D5002E
:1004F0008A150A1607208A110A12711C822A6024A2
:10050000BF00E524C82508000A30C8002C30CA0006
:10051000F218922A7219902A0030CA000330A02AD9
:100520000230A02A4927871D9E2A5030BD00871D12
:100530009E2ABD03031D972A0030A02A0130A02A5D
:10054000BC00831710308400831203133C08800022
:100550007015C82508001727642504270830C8002F
:100560002D30CA00C82508000830C8002E30CA0047
:100570008711412787113827071EC42A8A150A16B2
:100580009A228A110A12BB2A8715602560258711D5
:100590004927C82508000830C8002F30CA001A3083
:1005A000D500502D0830C8003030CA001930D500B1
:1005B000502D0830C8003130CA00F1248A110A16C3
:1005C000D2218A110A12F82408000830C8003230FB
:1005D000CA000D258A110A16D2218A110A1219257C
:1005E00008000830C8003330CA002608BC00250EB9
:1005F000BC0400303C02031DFF2A17270E2B0130DC
:100600003C02031D052B04270E2B02303C02031D68
:100610000B2BF1260E2B0630BF00E524C825080061
:100620000A30C8003430CA00831710308400B42662
:10063000831203131E08831203178000831203130F
:100640007015C82508000A30C8003530CA00831765
:1006500010308400F126B0261727831203131E08DA
:10066000831203178000831203137015C825080036
:100670000A30C8003730CA00831710308400B8260B
:10068000831203131E0883120317800083120313BF
:100690007015C82508000830C8003930CA000D257B
:1006A0008A150A16EB208A110A12F11C5A2B7016B1
:1006B0000730BF00192508000830C8003B30CA00C9
:1006C0002508BC0001303C0203196A2B0630BF002C
:1006D000E524742B8A110A16A7218A110A12711DAA
:1006E000742B0730BF00E524C82508000830C80077
:1006F0003C30CA00F801F901FA01FB01FC01FD01DF
:10070000FE01FF018A150A16EB208A110A124927F9
:10071000871D872B8E2B0730BF00E524C8250800D6
:100720001030C8003D30CA0070150D30D500502D76
:100730000830C8003E30CA00F1248A110A16D221BE
:100740008A110A12F8248A110A1208000830C80017
:100750003F30CA000D258A110A16D2218A110A12C9
:10076000192508000830C8004030CA00F1248A1159
:100770000A1631218A110A12F82408000830C8002C
:100780004130CA000D258A110A1692208A110A12D8
:10079000192508000830C8004230CA00C3248A1155
:1007A0000A16A7218A110A12C82508000830C800B5
:1007B0004330CA000D258A110A1612208A110A1226
:1007C000192508000830C8004430CA000D258A11D8
:1007D0000A1634208A110A12192508000830C800A8
:1007E0004530CA000D258A110A1671208A110A1295
:1007F000192508000830C8004630CA000D258A11A6
:100800000A164F208A110A12192508000830C8005C
:100810004730CA00F1248A110A16AE208A110A1242
:10082000F8248A110A1208000830C8004830CA00AB
:10083000F1248A110A16D3208A110A12F82408001A
:100840000830C8004930CA00F1248A110A16122162
:100850008A110A12F82408000830C8004A30CA0079
:10086000F1248A110A16F3208A110A12F8240800CA
:100870000830C8004B30CA002608C000250EC0044E
:10088000C82508000830C8004C30CA00C8256425B7
:10089000192608000830C8004D30CA00C825642554
:1008A000252608000030BF000A30C8000030CA000A
:1008B0008317103084003F0880007015C825080099
:1008C000F11D642C09306E2C711E682C10306E2CBA
:1008D000711F6C2C11306E2C08306E2C0800C32454
:1008E0008A150A1607208A110A12711C7B2C073000
:1008F000BF00E524902CC8255C257B3076255C253F
:10090000C9018A150A16BB218A110A124908E62074
:1009100039087625380876255C257D3076255C25D6
:10092000C8250800C3248A150A1607208A110A124E
:10093000711C9E2C0730BF00E524C12CC8257925E9
:100940007B3C0319A72C0130BF00E524C12CC90151
:100950008A150A16D2218A110A127925D620BC00DE
:10096000BC0E7925D6203C0449020319BA2C043068
:10097000BF00701679257D3C0319C12C0130BF00E2
:10098000E524C825080083132C08F8002B0EF80472
:100990002A08F900290EF9042808FA00270EFA049B
:1009A0002608FB00250EFB043408FC00330EFC0473
:1009B0003208FD00310EFD043008FE002F0EFE044B
:1009C0002E08FF002D0EFF0408000A30C80000307A
:1009D000CA0070158317103084003F088000061588
:1009E0000800C324C8255C257B307625C901080092
:1009F0004908E62039087625380876257D307625A1
:100A00000B2D0A30C8000030CA0070158317103053
:100A100084003F088000C82508007012C324C82540
:100A200079257B3C0319172D0130BF007016C901D1
:100A300008007925D620BC00BC0E7925D6203C04C0
:100A400049020319262D0430BF00701679257D3C1C
:100A500003192D2D0130BF00701603138312701E71
:100A60003B2D0A30C8000030CA00701583171030C3
:100A700084003F088000C8250800E6203908C9071F
:100A800076253808C907762508007925C907D620B4
:100A9000B900B90E7925C907D620B904390808006C
:100AA0008A150A1607208A110A12711C5A2D07305E
:100AB000BF00E524C8250800C8200B1D5D2D0800D7
:100AC000CE200B1D612D0800D1200B1D652D0800C7
:100AD000F300030E8301F5000A08F4008A0174088C
:100AE0008A00750E8300F30E730E0900F01C8A2D28
:100AF000AF2DF01C7C2D982D83120313F01A882D36
:100B000006148316891B852D822D83120610080872
:100B100006100800F01A972D83128C138800061413
:100B20008316091B912D83128C1F942D061008002B
:100B3000831203138C1AA02D86128C1AA02D9D2DC2
:100B40001A08AA2D1819A82D9818A82D0301AA2D46
:100B5000181218168616BA01BA0BAC2D0800C70079
:100B60000C1EB02D470899008316981CB52DB92D81
:100B700083128312080004304802C5008313213019
:100B80008400C9010008C907840AC50BC22D0800EA
:100B90008313203084005B308000840A4808E620FC
:100BA00039088000840A38088000840A4A08E62050
:100BB00039088000840A38088000840A701DFD2DE1
:100BC00008304802C5000310C50C2530C600831745
:100BD0001030F7008317770884000008E62083139D
:100BE0004608840039088000C60A840A3808800054
:100BF000C60A8317F70AC50BEA2DBB250330480246
:100C0000F6002030760784004908E6203908800085
:100C1000840A38088000840A5D3080004808C500D6
:100C200083132030840000087625840AC50B132E18
:100C3000080083120313861683164030990083122E
:100C400018121A081A0818160800831203138616B9
:100C5000831615309900831218121A081A081816EC
:100C600008008316D0308700A00005148514851570
:100C700004309F00831280309F0017278030CD0002
:100C8000C426080086157208CC0023278312031798
:100C9000103084006126840A6D26840A7926840A2D
:100CA0008226840A8F26031383124C08F2007218DE
:100CB000F126F218042772191727F2192327861133
:100CC000080003138312B42633301E02031C9D2E2A
:100CD0009A301E020318A12EA52E03138312B826E4
:100CE0006A081E02031C9D2E6C081E020318A12E0A
:100CF000A52E031383121727B026A4081E0203187B
:100D0000A12EA52E031383120427B42633301E020E
:100D1000031C9D2E9A301E020318A12EA52E03132C
:100D20008312F126B02617276A081E02031C9D2E87
:100D30006C081E020318A12EA52E83170130800017
:100D4000080083178030800008008317003080007F
:100D500008008317103084000030831780000800DB
:100D60009F121F129F11BC2E9F121F129F15BC2E87
:100D70009F121F169F15BC2E5F271F145F271F157C
:100D80001F19C02E1F100800031383128610113084
:100D9000CB00D0264D08CB00D02686146327080050
:100DA0000830BB00CB0D031CD72E8617D82E861318
:100DB0000000000000000000061700000000000016
:100DC00000000613BB0BD22E0800861406178617E8
:100DD0000800861406178613080086140617861363
:100DE00008000708D1005115D1145110510887008F
:100DF0007214F2107211F2118A110A12D1208A11A2
:100E00000A120B1D012F08000708D1005115D1103F
:100E10005114510887007210F2147211F2118A11E4
:100E20000A12D1208A110A120B1D142F080007087C
:100E3000D1005111D1145114510887007210F210D1
:100E40007215F21108000708D1005115D114511480
:100E5000510887007210F2107211F21508009412F6
:100E600083162016A012200887008312851608001A
:100E7000941283162016A01620088700831285126C
:100E8000080094128316A01120088700831205150C
:100E9000080094128316A0152008870083120511FC
:100EA0000800051281010B110B1D542F721208004E
:100EB000051681010B110B1D5B2F72160800BA017C
:100EC000BA0B602F0800CE200B1D642F08000030E5
:100ED000CF004F08CD00C426F126B02617276B0897
:100EE0001E020318782FCF0F692F0030CD00C426C3
:100EF0000800FF3FFF3FFF3FFF3FFF3FFF3FFF3F38
:100F0000FF3FFF3FFF3FFF3FFF3FFF3FFF3FFF3FF1
:100F1000FF3FFF3FFF3FFF3FFF3FFF3FFF3FFF3FE1
:100F20008207000010291C29522C242938294A291B
:100F30005C29682970297A298929A629522CBC297B
:100F4000BD29522CBE29C329522C522C522C522C72
:100F5000522C522C522C522CC929522C522CD629AC
:100F6000522C522C522C522CE329F029FD29082A0C
:100F7000132A1E2A292A342A442A842AAB2AB42A6C
:100F8000CB2AD22AD92AE52AF12A102B232B522C3C
:100F9000382B522C4B2B522C5C2B762B902B982BD6
:100FA000A62BB22BBE2BCA2BD62BE22BEE2BFA2B69
:100FB000062C142C202C2C2C382C422C4A2C522C55
:100FC000522C0800FF3FFF3FFF3FFF3FFF3FFF3F27
:100FD000FF3FFF3FFF3FFF3FFF3FFF3FFF3FFF3F21
:100FE000FF3FFF3FFF3FFF3FFF3FFF3FFF3FFF3F11
:100FF000FF3FFF3FFF3FFF3FFF3FFF3FFF3FFF3F01
:1010000008308A003E0882070034003400345F2B29
:101010007B2B912BD72BD82BD92BDA2BFF2B072C03
:1010200008308A003E088207003400340034112C56
:101030002F2C892C8A2C142D152D162DFF2B182DB5
:1010400008308A003E0882070034003400345F2BE9
:101050008A2B912B8A2B912B8A2BF72B8A2BFF34EF
:1010600008308A003E0882070034003400345F2BC9
:10107000832B912B832B912B832BED2B832BFF34F5
:1010800008308A003E0882070034003400340134FE
:10109000083401340434013404340134023401349A
:1010A0000234023408308A003E08820700340034DB
:1010B0000034013404340134043401340434013480
:1010C0000134013402340234992908308A003E0880
:1010D0008207003400340034152E352E5A2E672E28
:1010E000B42EB52EB62EB72EDB2E08308A003E0861
:1010F0008207003400340034192D1F2D202D212D9E
:10110000222D232D292D2A2D312D08308A003E082D
:1011100082070034003400343C2D512D692D702D90
:101120008F2D902D912D922D942D08308A003E0800
:101130008207003400340034952DB82DDD2DEA2DC2
:10114000EB2DEC2DED2DEE2D022E08308A003E0801
:10115000820700340034003400291C292E292F294D
:1011600047294829492957295829FF3FFF3FFF3F71
:10117000FF3FFF3FFF3FFF3FFF3FFF3FFF3FFF3F7F
:10118000FF3FFF3FFF3FFF3FFF3FFF3FFF3FFF3F6F
:10119000FF3FFF3FFF3FFF3FFF3FFF3FFF3FFF3F5F
:1011A000FF3FFF3FFF3FFF3FFF3FFF3FFF3FFF3F4F
:1011B000FF3FFF3FFF3FFF3FFF3FFF3FFF3FFF3F3F
:1011C000FF3FFF3FFF3FFF3FFF3FFF3FFF3FFF3F2F
:1011D000FF3FFF3FFF3FFF3FFF3FFF3FFF3FFF3F1F
:1011E000FF3FFF3FFF3FFF3FFF3FFF3FFF3FFF3F0F
:1011F000FF3FFF3FFF3FFF3FFF3FFF3FFF3FFF3FFF
:101200008A110A166D21DB006D21DC008A150A1295
:101210005522F121C008031D19298A110A12B4268A
:101220008A150A1276301E02031C192926231F2252
:101230001B29C7221F2208008A110A166D21DB0014
:101240006D21DC008A150A125522F121262319226C
:1012500039232D29C7221F221F2208001C29FF30F5
:10126000DB00DC005522F121C7221C221C2239237D
:101270008A110A166D21DB006D21DC008A150A1225
:101280005522F12126231C221C22392308001C2967
:101290002F298A110A166D21DB006D21DC008A15C9
:1012A0000A125522F121C7221F221F2208001C29E1
:1012B0008A110A166D21DB006D21DC008A150A12E5
:1012C0005522F12126231C2213238A110A12C82039
:1012D0008A150A1208006D29A122E008031D73294E
:1012E000DF08031979290130DF0203186C29E002B5
:1012F0006C2908007B22CA2108008E22CA2108001E
:101300007B22CA2108008A110A168E218A150A1228
:10131000871287118A110A12F1268A150A12790892
:10132000E0007808DF0021306006031998296B215E
:1013300008008A110A168E218A150A12871287114F
:101340008A110A12F1268A150A127908E000780833
:10135000DF0008008A110A168E218A150A128712E8
:1013600087118A110A12F1268A150A122F220C22DD
:10137000E0017808DF006B2108008A110A168E212F
:101380008A150A12871287118A110A1217278A15DD
:101390000A120800DD01DE018A110A1695218A155C
:1013A0000A12871587110830BB00871587110310B3
:1013B000871A0314DD0CBB0BD5290630BB0087153B
:1013C00087110310871A0314DE0CBB0BDF29DE0C18
:1013D000DE0C871587118A110A168E218A150A12CA
:1013E00008008712871587110830BB008716DB0CB1
:1013F000031C871287158711BB0BF6290630BB002B
:101400008716DC0C031C871287158711BB0B002A7B
:1014100087128715871108005C08E9005B08E8005F
:10142000FF30DC00DB00F1216908DC006808DB002C
:1014300008000130F700252A0230F700252A043081
:10144000F700252A1E30F700252A8A110A12CE201D
:101450008A150A120B1D2A2AF70B252A0800871263
:1014600087158711871287158711871287158711AE
:10147000871287158711871287158711871287159D
:10148000871108008716871587118712871587111E
:10149000871287158711871287158711871287157D
:1014A0008711871287158711080087128715871102
:1014B0008716871587118712871587118712871559
:1014C00087118712871587118712871587110800E2
:1014D0008716871587118716871587118712871535
:1014E0008711871287158711871287158711871231
:1014F00087158711080087128715871187128715AE
:10150000871187168715871187128715871187120C
:101510008715871187128715871108008716871589
:1015200087118712871587118716871587118712EC
:1015300087158711871287158711871287158711DD
:101540000800871287158711871687158711871658
:1015500087158711871287158711871287158711BD
:101560008712871587110800871687158711871638
:101570008715871187168715871187128715871199
:101580008712871587118712871587110800871220
:10159000871587118712871587118712871587117D
:1015A0008716871587118712871587118712871568
:1015B00087110800871687158711871287158711ED
:1015C0008712871587118716871587118712871548
:1015D00087118712871587110800871287158711D1
:1015E0008716871587118712871587118716871524
:1015F00087118712871587118712871587110800B1
:101600008716871587118716871587118712871503
:1016100087118716871587118712871587118712FB
:101620008715871108008712871587118716871578
:1016300087118716871587118716871587118712D7
:10164000871587118712871587110800871287155C
:1016500087118712871587118712871587118716BB
:1016600087158711871687158711871287158711A8
:101670000800871687158711871687158711871623
:101680008715871187128715871187168715871188
:101690008712871587110800871687158711871607
:1016A0008715871187168715871187168715871164
:1016B0008716871587118712871587110800203034
:1016C000F9000730F800AA217A21DE125E135E08C5
:1016D000DC005D08DB001925BD212030F900073052
:1016E000F800AA214222B422C7221F221F2242222E
:1016F000B422BD210800F801F901AA214C231F22C0
:101700001F22BD210800DA221F221F22C7221F220A
:101710001F22080000231F221F22C7221F221F2270
:10172000080083210430E800FF30E900A122E90B22
:10173000962BE80B942BA122A122A12280215D08E7
:10174000E5005E08E600BD21AA217A2166135E1A33
:101750006617E613DE1AE6172F220C22DA221F2262
:101760001F2200231F221F22BD2183210430E800F5
:10177000FF30E900A122E90BBA2BE80BB82BA1221C
:10178000A122A1226508DB006608DC006226BD21DB
:10179000AA217A215E12661B5E16DE12E61BDE1699
:1017A0005D08DB005E08DC002025BD2108007B2BE6
:1017B000912B7B2B2030F9000730F800AA2155220D
:1017C0000C22DA221F221F221F221F2200231F2287
:1017D0001F221F221F22BD210800832155220C2217
:1017E000DA221F221F221F221F22BD21080083216F
:1017F00000231F221F221F221F22BD210800F801E3
:10180000F901AA21DA221F222222BD210800AA21E1
:101810002F220C22DA221F221C221F221C22BD2171
:101820000800F801F90183214308E7004408E800B3
:101830001A2CA122FF30DB00DC005522F121C72247
:101840001F22E708031D272CE80803192D2C01305F
:10185000E8020318192CE702192CBD2108000330F7
:10186000F6004208E7004308E8004408E9000310D6
:10187000E70CE80CE90CF60B372CF901F801832191
:101880000830F600FF30DB00DC005522F121F60BBA
:101890004A2C4C2CA122422CC7221F221F22E708CF
:1018A000031D582CE808031D582CE9080319632C64
:1018B0000130E9020318612CE8020318612CE702E9
:1018C000612CA122402C2F220430E900FF30DB00E4
:1018D000DC005522F121C7221F221F22E90B712CA7
:1018E000732CA122662CA122FF30DB00DC005522E4
:1018F000F121C7221F221F22A122A122A122FF30F3
:10190000DB00DC005522F121C7221F221F22BD214E
:101910000800912BAE24F5248E240800F801F9016B
:10192000AA21FF30DB00DC005522F121C7221C2256
:101930001C2239230230E8000430E900A122FF30E4
:10194000DB00DC005522F121E90B9E2C26231C2212
:101950001C223923E80B9C2CBD2108000530F60021
:101960004208E7004308E8004408E9000310E70CD8
:10197000E80CE90CF60BB62CF901F8018321FF30D5
:10198000DB00DC005522F1212030DA000430F600C3
:10199000C7221C223923CF2C0430F600A122FF30AD
:1019A000DB00DC005522F121DA03F60BCE2C2623D6
:1019B0001C221C223923DA080319DF2CCC2CE7085F
:1019C000031DE82CE808031DE82CE9080319122D73
:1019D0000130E9020318F12CE8020318F12CE702A8
:1019E000F12CA122C42CBD2108001C221C22F901CB
:1019F000F8019921FF30DB00DC006822F121E901C8
:101A0000C7221C221C223923FF30DB00DC006822A5
:101A1000F12126231C221C221C221C223923A12254
:101A2000E90B002DBD210800912B8A2CDA2BFF2B0E
:101A3000FF345522F121C7221F221F220800192D31
:101A4000192D192D192D5522F121C7221C223923B8
:101A50000800192D5522F121C722C722192213236C
:101A600008005522F12126231C2213238A110A1271
:101A7000C8208A150A1208006822F121C008031D37
:101A80004D2D8A110A12B4268A150A1276301E02CA
:101A9000031C4D2D26231F224F2DC7221F22A122BA
:101AA00008006822F121C008031D642D8A110A1262
:101AB000B4268A150A1276301E02031C642D2623D2
:101AC0001F221F223923672DC7221F221F22A12276
:101AD00008006822F121C7221F221F22A12208002C
:101AE0006822F121C008031D832D8A110A12B42631
:101AF0008A150A1276301E02031C832D26231F220C
:101B00001F2239238D2DC7221C221C221C221C229D
:101B1000392326231C221C223923A1220800692DE7
:101B2000702D692D00340800FF348A110A166D21CA
:101B3000DB006D21DC008A150A125522F121E30A2F
:101B400059086306031DB72DC008031DB42D8A1163
:101B50000A12B4268A150A1276301E02031CB42D0E
:101B600026231F22E301B72DC7221F22E30108000D
:101B70008A110A166D21DB006D21DC008A150A121C
:101B80005522F121E30A59086306031DDC2DC00824
:101B9000031DD82D8A110A12B4268A150A12733031
:101BA0001E02031CD82D262319223923E301DC2D24
:101BB000C7221F221F22E30108008A110A166D2185
:101BC000DB006D21DC008A150A125522F121C722A3
:101BD0001F220800672EDD2DEA2DDD2D8A110A1641
:101BE0006D21DB006D21DC008A150A125522F121DE
:101BF000E30A59086306031D012EC7221922132385
:101C0000E30108008A110A166D21DB006D21DC005A
:101C10008A150A125522F12126231C2213238A1128
:101C20000A12C8208A150A1208008A110A166D21A4
:101C3000DB006D21DC008A150A125522F1210130EA
:101C400040020319302E8A110A12B4268A150A128C
:101C500076301E02031C302E26231F22E301342E71
:101C6000C7221F221F22E30108008A110A166D21D4
:101C7000DB006D21DC008A150A125522F121E30AEE
:101C800058086306031D592EC008031D552E8A11DE
:101C90000A12B4268A150A1276301E02031C552E2B
:101CA000262319223923E301592EC7221F221F227E
:101CB000E30108008A110A166D21DB006D21DC00AA
:101CC0008A150A125522F121C7221F220800C008D6
:101CD0000319A02E6B2EBD211922F901F8018321D1
:101CE000FF30DB00DC005522F121C7221C221C2220
:101CF00039230830E9008A110A166D21DB006D21B5
:101D0000DC008A150A125522F1210330E800A122D5
:101D10008A110A166D21DB006D21DC008A150A127A
:101D20005522F121E80B872E26231C221C22392361
:101D3000A122E90B7B2EFF01FE01FD01FC01B32E68
:101D40008A110A166D21DB006D21DC008A150A124A
:101D50005522F121E30A04306306031DB32E262326
:101D60001C223923E30108005A2E672E5A2E8A11AD
:101D70000A166D21DB006D21DC008A150A1255223E
:101D8000F121E30A8A110A1650218A150A128A15CE
:101D90000A12A1228A150A128A110A166D21DB0085
:101DA0006D21DC008A150A125522F121C722192261
:101DB0001323E30108008A110A166D21DB006D214F
:101DC000DC008A150A125522F121E30A26231C227F
:101DD00013238A110A12C8208A150A120800FF3F2D
:101DE000FF3FFF3FFF3FFF3FFF3FFF3FFF3FFF3F03
:101DF000FF3FFF3FFF3FFF3FFF3FFF3FFF3FFF3FF3
:101E0000FF3FFF3FFF3FFF3FFF3FFF3FFF3FFF3FE2
:101E1000FF3FFF3FFF3FFF3FFF3FFF3FFF3FFF3FD2
:1020000083171030840002308000840A073080007B
:10201000840A0130800008008317103084000130EA
:1020200080000800F1128A150A1240208A110A164F
:10203000D800E3018A150A1283218A110A16502159
:10204000003A03192E288A150A1265208A110A16E9
:102050008A150A12A1228A110A161F288A150A1245
:10206000BD218A110A160800F1128A150A1264208D
:102070008A110A165021003A031949286D21DB0004
:102080008A150A1285208A110A16DF0F3A28E00AFB
:102090003A288A150A12BD218A110A160800F1127F
:1020A000E3018A150A1252208A110A16D9008A15EC
:1020B0000A12AA218A110A165021003A03196B2824
:1020C0008A150A1295208A110A168A150A12A12267
:1020D0008A110A165C288A150A12BD218A110A166D
:1020E0000800F1128A150A12AA218A110A16502133
:1020F000003A03198C286D21DB006D21DC008A1564
:102100000A1275208A110A16DF0ADF0A8A150A12D6
:10211000A1228A110A1677288A150A12BD218A116E
:102120000A160800F112E3018A150A12AA218A117F
:102130000A165021003A0319A8288A150A12A52068
:102140008A110A168A150A12A1228A110A169928DA
:102150008A150A12BD218A110A160800F1128A1581
:102160000A1283218A110A165021003A0319CD2838
:102170008A150A1280218A110A165D088A110A122C
:102180003D255E088A110A123D258A110A168A1514
:102190000A12A1228A110A16B4288A150A12BD2130
:1021A0008A110A160800F1128A150A1264208A118F
:1021B0000A165021003A0319ED288A150A127D21CA
:1021C0008A110A165D0873218A150A12A1228A1142
:1021D0000A16DF0FD928E00AD9288A150A12BD216C
:1021E0008A110A160800F1128A150A12AA218A1108
:1021F0000A165021003A03190C298A150A12802167
:102200008A110A165D0873215E0873218A150A1265
:10221000A1228A110A16F9288A150A12BD218A11EB
:102220000A160800F1128A150A12AA218A110A1642
:102230005021003A03192B298A150A127A218A1192
:102240000A165D0873215E0873218A150A12A122FD
:102250008A110A1618298A150A12BD218A110A162E
:102260000800F1128A150A12AA218A110A165021B1
:10227000003A03194A298A150A1280218A110A167E
:102280005D0873215E0873218A150A12A1228A1142
:102290000A1637298A150A12BD218A110A16080062
:1022A0008A110A16FF08031D5E29FE08031D5E2918
:1022B000FD08031D5E29FC08031900340130FC02EF
:1022C00003186929FD0203186929FE020318692908
:1022D000FF02FF308A110A1608008A110A124525EA
:1022E0008A110A1608008A110A123D258A110A1657
:1022F00008008A110A12B4268A110A1676301E02C4
:10230000031C85298A150A1200288A150A1210282A
:102310008A150A1230288A150A1220288A110A12F0
:102320002F2741278A110A1608008A110A12382716
:102330008A110A1608008A150A1262288A150A12DA
:1023400063288A150A1250288A150A1251288A1100
:102350000A1608000130E40008000230E40008001A
:102360000230E4000800831203133830EA00C12170
:10237000EB00AF30EC008A110A1267278A110A16A7
:10238000D12911308A003E0882070034003400341D
:102390009C349C349C349C349C349C349C34A234B7
:1023A0009C3408000034FF3FFF3FFF3FFF3FFF3FEB
:1023B000FF3FFF3FFF3FFF3FFF3FFF3FFF3FFF3F2D
:1023C000FF3FFF3FFF3FFF3FFF3FFF3FFF3FFF3F1D
:1023D000FF3FFF3FFF3FFF3FFF3FFF3FFF3FFF3F0D
:1023E000FF3FFF3FFF3FFF3FFF3FFF3FFF3FFF3FFD
:103000000313831600309400831294120800831275
:1030100003130130550603195A28023055060319C7
:1030200066280330550603196D2804305506031928
:103030007F280530550603199128063055060319D7
:103040009D28073055060319A9280830550603198D
:10305000B528093055060319C1280A305506031949
:10306000D3280B3055060319E5280C3055060319F3
:10307000EB280D305506031929290E305506031982
:10308000632918305506031970291930550603199C
:103090007D291A30550603197F291B30550603195F
:1030A00081291C305506031982291D305506031944
:1030B00094290800A621711865281D228317103055
:1030C000840056088000831203130800A62171189B
:1030D0006C280330D200E7210800A62171187E2851
:1030E0008A110A16A121D2008A150A16F1218A1125
:1030F0000A16A421D2008A150A1607220800A62162
:10310000711890288A110A16A121D2008A150A1670
:10311000F1218A110A16A421D2008A150A16072263
:103120000800A62171189C288A150A16D200F121E0
:103130008A150A16D20007220800A6217118A828AD
:103140008A150A16D200F1218A150A16D200072222
:103150000800A6217118B4288A150A16D200F12198
:103160008A150A16D20007220800A6217118C02865
:103170008A150A16D200F1218A150A16D2000722F2
:103180000800A6217118D2288A110A169B21D200A4
:103190008A150A16F1218A110A169E21D2008A1573
:1031A0000A1607220800A6217118E4288A110A16B7
:1031B0009B21D2008A150A16F1218A110A169E2136
:1031C000D2008A150A1607220800A621D701721B11
:1031D000D70A45220800F110831203137C08D70098
:1031E0004522F119F1147D08D7004522F119F11497
:1031F0007E08D7004522F119F1147808D70045223E
:10320000F119F1147908D7004522F119F1147A085F
:10321000D7004522F119F11416298A110A12452501
:103220008A150A16D7004522F119F114FE08031D6C
:103230001F29FD08031D1F29FC0803192829013037
:10324000FC0203180D29FD0203180D29FE020D29A9
:103250000800A621711862298A110A169E21D2003F
:103260008A150A168317103084008001840A8001B1
:10327000840A8001840A8001E721831710308400CA
:10328000840A840A840A0008D400103084000008EC
:10329000840A840A840A8000103084005408800064
:1032A000831710308400840A840A0008D400103088
:1032B0008400840A0008840A800010308400840A94
:1032C000540880000800A62171186F297808D700DB
:1032D00045227908D70045227A08D7004522080000
:1032E000A62171187C297808D70045227C08D700D0
:1032F00045227D08D70045220800A6210800A62106
:1033000008000800A6217118D2288A110A16D221B5
:10331000D2008A150A16F1218A110A16D221D2008A
:103320008A150A1607220800A6217118E4288A11B6
:103330000A16D221D2008A150A16F1218A110A161C
:10334000D221D2008A150A160722080071105508EA
:10335000D7004522711B7114FF30D6001D22711A4F
:10336000711456085702031D7114D608031DBA299B
:1033700071141D2208008A110A1650218A150A1696
:10338000003A0319D1296408D2001D22711AD129EB
:1033900056088A110A123D258A150A16D20BC5292C
:1033A000BB2908008A110A1650218A150A16003A0C
:1033B0000319E6296408D2008A110A1245258A15E4
:1033C0000A16D7004522D20BDC29D2290800831720
:1033D000103084001D2256088000840AD20BEA298E
:1033E00008007808D7004522D2030319062A790875
:1033F000D7004522D2030319062A7A08D7004522AE
:10340000D2030319062A7B08D700452208007C084E
:10341000D7004522D20303191C2A7D08D700452274
:10342000D20303191C2A7E08D7004522D2030319B0
:103430001C2A7F08D7004522080071126D22F1195D
:103440003D2A8A110A1238278A150A169301253057
:10345000940094168C110A30D3008A110A12D120DC
:103460008A150A160B19372A8C1D322A3A2AD30BD1
:103470002D2A3D2A1308D6003E2A711687128A117A
:103480000A122F278A150A1608006D22F1195E2AE2
:1034900071132530940094168C11570893000A304C
:1034A000D3008A110A12D1208A150A160B195B2A39
:1034B0008C1D562A5F2AD30B512A5E2A71178A1156
:1034C0000A12CB208A150A160B1D642A87128A114C
:1034D0000A122F278A150A160800F1118A110A12FA
:1034E000492787128A110A122F278A150A16643073
:1034F000D3008A110A12D1208A150A160B19832AC1
:10350000871D7E2A862AD30B792A982A8A110A12C5
:10351000C8208A150A160B1D8B2A87168A110A12D3
:10352000D1208A150A160B19982A8719932A992AE5
:10353000F11508008A110A12492738278A150A1638
:10354000D601071EA12A871DA32A0830D300871D94
:10355000A72A8719A92A0310071A0314D60DD30B1B
:10356000A72A871DB12A8719B32ADA228A110A12DB
:1035700041278A150A168715000000000000000088
:1035800087118A110A12492738278A150A16080056
:103590008A110A12D1208A150A16E02A8A110A1203
:1035A000CE208A150A16E02A8A110A12CB208A1523
:1035B0000A16E02A8A110A12C8208A150A16E02A79
:1035C0000B1DE02A0800003400340002000700014F
:1035D000FF3FFF3FFF3FFF3FFF3FFF3FFF3FFF3FFB
:1035E000FF3FFF3FFF3FFF3FFF3FFF3FFF3FFF3FEB
:1035F000FF3FFF3FFF3FFF3FFF3FFF3FFF3FFF3FDB
:10360000FF3FFF3FFF3FFF3FFF3FFF3FFF3FFF3FCA
:1038000083120313FB308605083086041030BE0097
:1038100020308400B02580003C302002031D0A2C9B
:10382000840ABE0B0A2CC3010C30BE002130840078
:103830000008C307840ABE0B182C0A30BE002530CE
:1038400084000008C1258000840ABE0B212C2808B2
:10385000B900270EB9042608B800250EB8042C08B4
:10386000BD002B0EBD042A08BC00290EBC0438087C
:10387000BA003908BB003D08BB07031C402CBA0A3C
:103880003C08BA073C302002031DBB2C3E302F02FF
:10389000031DBB2C2E08F5002D0EF5044308750200
:1038A000031DBE2C1B303A020319592C031C602C3B
:1038B000C12CFF303B020319602C0318C12C602C73
:1038C000003038020319672C03186D2CC12C04300A
:1038D000390203196D2C031CC12CC724B025A0008C
:1038E0007B302002031DBB2CC3013808F4003908CB
:1038F000F300F501F6010430BE0020308400B0254D
:10390000C307C1258000840ABE0B7F2C2308F60064
:10391000220EF6042108F500200EF504FF24000015
:103920000000000000000000000000000000000097
:10393000F30A0319F40A3A087402031D792C3B08B0
:103940007302031D792CB025C125A000B025C12527
:10395000A100200EA10443082102031DBE2CB025A6
:10396000A0007D302002031DBB2C83120313F7300F
:103970008605C724BA2C3130D824692D3430D82498
:10398000692D3630D824692D3730D824692D5B3025
:10399000AA253030AA253830AA253130AA25303062
:1039A000AA254330AA253930AA255D30AA2508006A
:1039B000F500B025A0007D3020020319E42C3E3034
:1039C00020020319E42CD92C5B30AA253030AA251B
:1039D0004130AA253030AA253030AA253030AA251A
:1039E0007508AA253330AA25750AAA255D30AA25AF
:1039F00083120313F730860504308604080003178A
:103A0000831273088D0074088F0075088C00760887
:103A10008E0083168C170C158B1355308D00AA3031
:103A20008D008C14000000000C1103138312080099
:103A30000317831273088D0074088F0083168C1788
:103A40000C140000000083120C08F7000E08F800A8
:103A5000031308008312031386168316403099005F
:103A6000243098008312903098001A081A087010B9
:103A70000800831203138C1A472D81010B11861243
:103A80008C1A472D7018402D0B1D402D492D1A08FA
:103A9000512D18194F2D98184F2D0301512D181223
:103AA00018168616BF01BF0B532DBF010800031364
:103AB0008312061A592D8316981C5C2D83129900C7
:103AC000080083120313D1256625692D2A25E925CF
:103AD00008007010B025F900553079020319812DC6
:103AE000563079020319922D5A3079020319962D16
:103AF000503079020319A42D463079020319A72DFD
:103B0000692D7014F01C852D872D18128A2D8316AF
:103B1000091283128312031306117530AA258A0134
:103B20001030820070147630AA25002C7014831295
:103B3000031306110130AA250130AA250130AA2558
:103B40000330AA257010692D86150611A62D0615BD
:103B50008611A92DF01CAE2D5725AF2D0526080086
:103B6000701CB92DF01CB72DB52D3925C02DF125B0
:103B7000C02DF018BC2DBE2DF010B72DF014B52DB2
:103B80000800FA00F9000F30F90547307A020318EF
:103B9000CF2D41307A02031CCF2D0930F907790867
:103BA0000800031383160B30850010308600903018
:103BB00087001730890004309F008312033087008C
:103BC00000308600103085008316D63081008312C5
:103BD000080003138316173089008312031306109D
:103BE0000800831203133D3081000B110614831665
:103BF000891B002E7018F72D0B1DF72D0301032EC6
:103C000083120610080806100800831203138800A8
:103C100006148316091B0A2E831206100800FF3FA4
:103C2000FF3FFF3FFF3FFF3FFF3FFF3FFF3FFF3FA4
:103C3000FF3FFF3FFF3FFF3FFF3FFF3FFF3FFF3F94
:103C4000FF3FFF3FFF3FFF3FFF3FFF3FFF3FFF3F84
:103C5000FF3FFF3FFF3FFF3FFF3FFF3FFF3FFF3F74
:02400E00723FFF
:08400000FF3FFF3FFF3FFF3FC0
:00000001FF
